:100000006F00403D0000000032010000340100009C
:1000100000000000000000000000000000000000E0
:1000200000000000000000000000000000000000D0
:10003000D203000000000000D20300000000000016
:10004000D2030000D2030000D2030000D20300005C
:10005000D2030000D2030000D2030000D20300004C
:10006000D2030000D2030000D2030000D20300003C
:10007000D2030000D2030000D2030000D20300002C
:10008000D2030000D2030000D2030000D20300001C
:10009000D2030000D2030000D203000000000000E1
:1000A000511126C022C206C4828282441244A24058
:1000B00031018280634E050263C305042E86AA8542
:1000C0007D5515C285466378B6006356C0000606A6
:1000D0008606E36CB6FE014563E4C500918D558D3F
:1000E00085820582F5FA82808682C93F2E858282CA
:1000F0003305A04063D70500B305B040C1B7B305D1
:10010000B0408682653F3305A0408282868263C705
:100110000500634905005D372E858282B305B04036
:10012000E35B05FE3305A040513F3305B0408282BA
:10013000000001A001A0EFF2BFF611651111854585
:100140001305050202C002C202C402C602C802CAE6
:1001500002CC7129930700027C80371401408D473F
:100160003EC28A85E147130504403EC4ED2C930747
:1001700000047C808A859147130504403EC4E52431
:10018000F16737440140938707203EC66C00B707EC
:100190000C00130504803ECA02C8231C0100BD21C7
:1001A0008545130504801D23710101B7EFF25FEF50
:1001B000054569265D2A9923716513050520BD2330
:1001C000B707002083A5070137150000130545D8A0
:1001D000EF0010396124AA8537150000130545D9B1
:1001E000EF001038893FB7040020374401409307DF
:1001F00004803E8593050002ED29B74701409387AF
:10020000078065D913050480CD2193878403137576
:10021000F50F88A38C23130504803744014093C550
:10022000F5FFC205C18175291304048093050008F8
:100230002285C12165DD55BFEFF29FE637140240EC
:100240001C403707FFFC611193E717001CC05C409E
:100250004145F98F5CC01C403707F7FE7D17F98FC9
:100260001CC01C403707FCFF7D17F98F1CC05C4089
:1002700041777D17F98F5CC0B7079F001CC4E1244C
:100280001C4C3706020093E707021CCCB71701404D
:1002900003A70740938607401377F7F023A0E740B2
:1002A00003A707401367070823A0E74089479CCAB4
:1002B00002C002C21C4C37070140A16693E7170039
:1002C0001CCC5C43D58F5CC31C404167B716024011
:1002D000D98F1CC009679C42F18F3EC282478507B7
:1002E0003EC0924781E78247E397E7FEB717024097
:1002F0009C431397E7006358070685473EC21247A1
:1003000085476310F706B72702409843C176FD166C
:10031000719B98C398431367170098C3B71702409F
:10032000D843D8C3D843758FD8C3D843C166558F37
:10033000D8C39843B7060001558F98C398439316C6
:100340006700E3DD06FED843B7160240719BD8C3B1
:10035000D84313672700D8C32147DC42B18BE39E03
:10036000E7FE210199B302C259BFEFF27FD33717DD
:1003700002405C43370400209146B18B1304040112
:100380006385D700A1466380D704B7376E01938792
:1003900007601CC0B7160240DC420840918313F787
:1003A000F700B707002093870700BA978C23DC4239
:1003B00093F5F50F93F707083357B50099E3FD3927
:1003C0002A8718C0DDB15C43B777DC02938707C08A
:1003D000C9B701A09701002093814146138181FC98
:1003E000171500001305C59C97050020938585C14E
:1003F00017060020130686C463FAC5008322050091
:1004000023A0550011059105E3EAC5FE170500205C
:100410001305C5C29385C1806377B500232005000D
:100420001105E36DB5FEB722000093820288739038
:1004300002308D427390428097020000938282BC0A
:1004400093E2320073905230EFF01FDF970200000A
:10045000938202D67390123473002030B7F7FF1FD7
:1004600003A5477C82809C45611122C226C013F7F8
:10047000070113F3F70001C7D8413363E30092216A
:100480001377F60F29C78323050001471304800261
:10049000930480048546B395E600B376B600639274
:1004A000D50293122700BD46B396560093C6F6FFB9
:1004B000B3F37600B3125300B3E372006397870679
:1004C0004CC90507A146E317D7FC23207500130785
:1004D000F00F6378C70483234500A146130480020C
:1004E000930480040547B312D70033775600639412
:1004F000E202139726000117BD45B395E50093C5A9
:10050000F5FFB3F375003317E300B363770063922D
:100510008702232A550085064147E395E6FC2322FE
:1005200075001244824421018280E39C97F80CC933
:1005300049BFE39297FE23285500F1BFB70700207B
:1005400023AEA7028280371702401C430E0593F7A3
:1005500077F05D8D08C38280EFF29FB437170240B9
:100560005C4391462A84B18B6385D700A146638A98
:10057000D706B7376E01938707601CC0B7160240D5
:10058000DC42918313F7F700B707002093878702B7
:10059000BA978C23DC42184093F5F50F93F70708C0
:1005A0003355B70099E33A85113E48C008C448C4A2
:1005B000B7170240DC43AD83FD8B13D737008A07A2
:1005C000F18BD98F93F637010D476373D700D1179D
:1005D0003707002013074701BA978C23C53408C892
:1005E000E9B45C43B777DC02938707C079B799C554
:1005F000371702401C4F5D8D08CF8280B71702402D
:10060000984F1345F5FF798D88CF8280EFF25FA96F
:100610001629F577FD17F58FF621DA252111D58FEB
:100620001EA95625FD779387379FF58FD6212A84FB
:100630002EC0D58F9625D58FB625D58F5EA55E2980
:10064000C207C18393F7F7CF5D8F5AA948002937B6
:10065000B7470140938707808245631DF404C24772
:100660005A24139517003E9542070E0541873E9583
:100670008C416353070486059134930540062AC0D4
:10068000353C824793144500930540063E85A93CBE
:100690005E24C207C18763D307020E059305400697
:1006A00013052503213C1D89C98CC204C18006A401
:1006B0006101E5BAB2476DB78A057DBF12059305A2
:1006C000400613052503DD3A3D89F9BF91C55E2536
:1006D0000967D98F5EA582805A25F977FD17F98FB2
:1006E000D5BF93F5F51F4EA182804A211375F51FE2
:1006F00082800A216D8D3335A0008280EFF25F9AEF
:10070000B707002003A50701B7157A0093850520D8
:1007100075321375F50F2385A18093175500898FC6
:100720008A073E950E052394A18041B2EFF25F97B0
:100730002A84116511118545130505024D3D930766
:1007400000027C80371501408D473EC28A85E14713
:10075000130505403EC4013B22C637440140B7079C
:1007600008006C00130504803ECA02C8231C010067
:10077000713D854513050480913F71013DB2EFF253
:100780003F927111AE840144635DC402B7470140DA
:10079000138707803A859305000432C0993FB74715
:1007A000014013870780024675D53387840083058F
:1007B0000700138507800504C205C1811D37024665
:1007C000E1B7328511016FF05F8E411106C62EC070
:1007D0000DCD1841AA8705C358417D5511CB8546DB
:1007E000631BD70098472300070023A20700054595
:1007F000B240410182809847824614A3984705077A
:1008000098C7D8437D17D8C3DDB705468A85853F8D
:10081000F9BF011122CC2EC206CE26CA2A848147F6
:1008200093050002634506029245BE958385050047
:100830008DE563D8C70263D4E702198E1305000261
:1008400093F526002AC089C501E7930500032EC051
:10085000858A814495EAB2840DA08507F1B71D8E83
:10086000F1BF0146E1BF824522853AC832C63EC487
:10087000A93FA24732464247FD14E34690FEB284A8
:10088000635306008144058E63C7E702A68792463C
:100890003387974036978305070095EDB28463440C
:1008A0009004635306000146F2406244D24433058B
:1008B000F600056182801D8FBA87930500032285AB
:1008C00032C83EC63AC41137B24722474246FD17E6
:1008D000EDF7BA9465BF228532C63EC4FD35A24706
:1008E000324685076DB78245228532C43EC2F13D4E
:1008F000FD142246924765B7397106DE22DC26DAFE
:100900003EC232833A8689ED92469307000301473F
:100910006C08FC86FD3DF2506254D2542161828005
:10092000AA843684AE8791CA294701446317E3003D
:1009300063D50500B307B04005448646A30901020C
:1009400013073103938666FC36C49A853E8532CA06
:100950003AC81AC63EC0EFF02FF9A5468247324387
:100960004247524663D4A600A246369513050503B6
:100970009306F7FFA30FA7FE9A853E8532CC3ACAAD
:100980001AC83EC636C0EFF06FF3B2474243524733
:10099000624663F9670401CC29CA9247898BB1C7C3
:1009A0009305D002268532C40D3522467D16924726
:1009B000918B95C306479307100632C49305000335
:1009C0002685631EF7021135930580072685F53BC2
:1009D0002246090479161647924682452685153D1A
:1009E000229515BFAA8702478DB782469307D0028A
:1009F0000144A38FF6FE9307E7FF3EC04DBFF133DE
:100A000093058005E1B7014582800145828013018D
:100A100081FD22D026CE06D22AC4AE82328402C6FE
:100A200081448385020089EDA24781C781453E85C7
:100A3000693B925002542685F24413018102828060
:100A4000930750026388F500224516C88504B53B1C
:100A5000C24239A88387120013871200639CB70033
:100A60002245930550023AC88D3342478504BA8225
:100A7000850245BFD5DB9306B0026389D70463C8FE
:100A8000F600930630026386D704814705A09306DB
:100A9000D002638AD70093060003E398D7FE13873A
:100AA0002200894721A0138722008547830607007B
:100AB0001306B0026383C6046341D60213063002F4
:100AC000638BC602BA820145A54681A01387220026
:100AD0006DBF138722009147D1BF1306D0026389EF
:100AE000C60013060003E39FC6FC93E7270031A06E
:100AF00005078547C1BF93E747000507E1B7131610
:100B00002500329506053A958502038602001307F3
:100B100006FD9375F70FE3F4B6FE1307E00299465E
:100B2000631EE60085028146A54503860200130682
:100B300006FD1377F60F63F5E50236C6038702005C
:100B40001306A006630DC70A6343E6021306C0043A
:100B50006307C70A13068006630CC70881452DA8E2
:100B600013972600BA968606B29685027DBF1306B5
:100B700040076306C7081306A0076302C7081306E9
:100B8000C0068145631AC700038612008D456314B1
:100B9000E600850291458502038602009303000664
:100BA0001307100663C4C3001307100493037006F1
:100BB00063C4C3069303500663537618930370040B
:100BC00063C1C30493055004635BB6161307300476
:100BD000E310E6EA18409303440016CA230CE10030
:100BE0001EC8A30C01000147BE862A862C0849A80E
:100BF000038612008145E311E6FA890271BF85027E
:100C0000B1BF93063006E307D6FC63CEC606930653
:100C100080056303D602A9BD930630076304D6049A
:100C200063CBC6029306F0066302D60E9306000756
:100C300093E74700E31ED6E29146639FD50A9303EC
:100C400084000C40504016CA3AC23EC01EC8AA8753
:100C50000147C146B9A0930650076308D60693061C
:100C6000800745BF1840B7160000930344009385E2
:100C700046DA11C3BA85324716CA1EC8BE862A860E
:100C80002245413E0DA091466394D5029303840012
:100C90000C40504016CA3AC23EC01EC8AA8705473B
:100CA000A94622458D33C243AA941E84D242C9B3B9
:100CB000B2460C4016C836C23AC011042A8785468F
:100CC000294622451539AA9461B39146639DD50002
:100CD000930384000C40504016CA3AC23EC01EC85E
:100CE000AA87014775BFB2460C4016C836C23AC043
:100CF00011042A878146E9B7B24616C80C4041461E
:100D000036C23AC011042A87814665BF9146639E68
:100D1000D500930384000C40504016CA3AC23EC02E
:100D20001EC8AA870147A146ADBFB2460C4016C8EF
:100D300036C23AC011042A878146214659B70C4071
:100D40001306840040403AC22A87224532C83EC07A
:100D50002286B687A94616CA4D39AA944244B9B725
:100D60001301C1FD2EC832CAAA851008014506C666
:100D700036CC3ACE3ED032C05939B240130141028E
:100D80008280000053797374656D436C6B3A2564FF
:100D90000D0A00004368697049443A253038780DDF
:0C0DA0000A000000286E756C6C29000031
:100DAC0001020304050607080102030405060708EF
:100DBC00006CDC020204060804080C100810182051
:100DCC001020304020406080010203040506070813
:080DDC000102030405060708EB
:00000001FF
